:10000000830100308A002428F60003088301CA0017
:100010008B1A0B1D1D280B11F03083120313810066
:10002000AB0AA11C1728AC0A031D1728A115211D16
:100030001D28AD0A031D1D282116031383124A082B
:100040008300F60E760E09002230840048303120FD
:1000500020308400223031208301F92C04068001F5
:10006000840A0406031D2E28003483120313C800DB
:10007000C91B4328491B4B2849088A004808C80A5D
:100080000319C90A82008313491883174808C80A4C
:10009000840000080800FC34FE34073403340334C1
:1000A000033403340734FE34FC340F341F34383443
:1000B000303430343034303438341F340F3400347A
:1000C00008340C340E34FF34FF3400340034003470
:1000D000003400340034303430343F343F34303472
:1000E0003034003400340C340E3407340334033419
:1000F0008334C334E7347E341C34303438343C34F5
:100100003E343734333431343034303430340C34DA
:100110000E34073403340334C334E734F634BE34C6
:100120001C340C341C3438343034303430343034F3
:1001300039341F340F34FF34FF34C034C034C0347A
:10014000C034C034C034FF34FF34003400340034D1
:10015000003400340034003400343F343F347F3402
:100160007F3463346334633463346334E334C334DB
:10017000833430343034303430343034303430340C
:1001800038341F340F34FC34FE34C73463346334E2
:1001900063346334E334C73486340F341F34383463
:1001A000303430343034303438341F340F34033486
:1001B000033403348334C334E33473343B341F34A3
:1001C0000F343C343E3407340334013400340034FB
:1001D0000034003400341C34BE34F73463346334E8
:1001E00063346334F734BE341C340F341F34393471
:1001F000303430343034303439341F340F343C34FC
:100200007E34E734C334C334C334C334C734FE3418
:10021000FC340C341C343834303430343034303422
:1002200038341F340F34C034C034C034C034C03408
:10023000C034C034C034C034C0340034003400345E
:10024000003400340034003400340034003400340E
:1002500000340034003400340034003400340034FE
:1002600000340034003400340034003400340034EE
:1002700000340034003400340034003400340034DE
:1002800000340034003400340034003400343C3492
:100290003C343C343C34003400340034003400340A
:1002A0000034003400341E343F34333433343F34AC
:1002B0001E34003400340034003400340034003480
:1002C000003400340034F834FC340E340734033482
:1002D0000334033407340E340C3407341F341C3415
:1002E000383430343034303438341C340C348207F1
:1002F000C0347E3441347F34C034383444344434E0
:10030000443438347C340834103408347C340834B1
:10031000083408340834083427344834483448341E
:100320003F3440343834043404347C347C34203456
:10033000103408347C347C34403440347C34C03451
:100340002034543454345434783400340034003479
:10035000003400347F3408341434223441342234DD
:1003600049344934493436343E34413441344134DB
:100370003E347F3445344534453439347F34093490
:100380000934093406347F344834303400347F343F
:100390007F3449344934493436343E34413441346D
:0E03A000413422347C341034103410347C3458
:1004FC0002308301BE00BE0B812A0800123083013A
:10050C00BE00BE0B872A08008A308301BC00BC0BDE
:10051C008D2A08009E308301BC00BC0B932A080076
:10052C008301C400861686104123861408008301BB
:10053C00C000861286104123861408008301BF0078
:10054C003E08073940389D223F087F3980389D2A64
:10055C0083012B08BD001930BD072B083D02BC00E0
:10056C00BC08031908006400B32AF401F501031058
:10057C00F30CF20C031CC92A7008F4077108031859
:10058C00710AF5070310F00DF10D720873040319CD
:10059C000034BD2A8301BE010030A422F830BC0017
:1005AC000130BD00640000309622BC080319BD0365
:1005BC00BC033D08803AF000803070020130031912
:1005CC003C02031C0800D82A08308301BC00BD0182
:1005DC0064000512831605120000000000000516C9
:1005EC007E222011051A201584220310BD0C201D1B
:1005FC00012B8030BD077E22BC0BEE2A7E223D08EB
:10060C000800073083019F0086018501FF308316A7
:10061C008500C430860020308B0083128C01831639
:10062C008C0107308100F030831281008B17A013EE
:10063C00A111A110211021122111080008308301F1
:10064C00BC00BD01640006118316061100000000F9
:10065C00000006157E22A0100619A0148422031097
:10066C00BD0CA01C3B2B8030BD077E22BC0B282B65
:10067C007E223D0808008301C50064000830C600D6
:10068C00C7010612C51F4C2B06144D2B061006165F
:10069C000310C50DC6080319C703C6034708803AE3
:1006AC00F00080307002013003194602031C080070
:1006BC00472B6400831203138615861400008611E1
:1006CC00AE22861521309D2245309D22C8309D22B8
:1006DC0006309D2214309D2220309D2209309D220F
:1006EC00D02208309D220C309D22BE010030A42A5D
:1006FC008301BC00C100C2010530BF00C001013044
:10070C008A0041087721BD00BE019622C10A031957
:10071C00C20ABF080319C003BF034008803AF000A7
:10072C0080307002013003193F020318852B003012
:10073C00962A8301BC000830BD0020113C182015FE
:10074C00831203130512831605120000000000002B
:10075C0000008312201DB52B83160516B72B8316AC
:10076C0005128422831605167E220310BC0CBD0BC9
:10077C00A32B7E2A8301BC000830BD00A0103C18BE
:10078C00A014831203130611831606110000000037
:10079C00000000008312A01CD62B83160615D82B44
:1007AC00831606118422831606157E220310BC0CB8
:1007BC00BD0BC42B7E2A83013C08C2003D08C3003C
:1007CC000A30C000C1014308003EC90042084B3E3C
:1007DC000318C90A3520BE00BF019622C20A0319AC
:1007EC00C30AC0080319C103C0034108803AF000D2
:0407FC0080307002D7
:100800000130031940020318E92B00309622003012
:10081000962A640083120313A301A201831605160E
:100820000615831205120611831605120611902271
:100830008316051606158422A0110619A015831229
:1008400003132012051A20168A22A0120619A016D8
:10085000831203132013051A2017A01A312CA201AA
:10086000A20A201B352CA301A30AA01D392C02309B
:10087000A207201E7E2A0230A3077E2A8301BD0024
:100880003C08BA00BB01BB00BA013D08BA04BB1F5B
:10089000592C20143B08F1003A08F000F009F10946
:1008A00001307007BA000030031801307107BB0037
:1008B0005A2C20100530F200F3013B08F1003A08F1
:1008C000F000BB227408AE007508AF002F0DAF0C0E
:1008D000AE0C2F0DAF0CAE0C2F0DAF0CAE0CA50156
:1008E000A401A6012E08B8002F08B9003908803AE3
:1008F000F000803070020A3003193802031CAB2C60
:10090000F630380739080318390AFF3E8039031DCD
:100910008E2CA60AF630B807031CB9032608F0008F
:10092000F101F63E71080318710AFF3E8039031D7C
:100930009C2CA40AF630A6072408F000F101F63E2C
:1009400071080318710AFF3E8039031D762CA50A31
:10095000F630A407762C3808B6003908B700260808
:10096000B400B5012408B200B3012508B000B101FC
:10097000201CBD2C0A30B000B101A508031D0800E1
:10098000A408031DEF2CA608031DE42C3908380425
:10099000031DD72C0B30B400B501B2003508B300ED
:1009A0003208B0003308B100B601B7010800201CBE
:1009B000DB2C0A30DC2C0B30B200B3010B30B00062
:1009C000B101B401B5010800201CE82C0A30E92C63
:1009D0000B30B200B3010B30B000B1010800201C95
:1009E000F52C0A30B000B10108000B30B000B101A5
:1009F0000800640007235F23BE01BE0A0030A42262
:100A00000F307E230F307E230F307E230F307E2366
:100A10002D307E2355307E2328307E2319307E23CF
:100A200005307E235A307E232D307E230F307E23E7
:100A30000F307E230F307E230430BE000030A4220E
:100A40000F307E230F307E230F307E230F307E2326
:100A50002D307E2314307E2319307E231E307E23DA
:100A600023307E2328307E232D307E230F307E23BB
:100A70000F307E230F307E238B1309248B17220324
:100A800003195F2E2208023A0319272E8B13CC304C
:100A9000C0238B17A118532D8B134430C0238B1701
:100AA000A114AC01A111A118061D5D2DA11D5D2D84
:100AB0008B13BE30C0238B17A017AE22A01F9F2E12
:100AC0008B132423A7002423A9008B17BC0027081D
:100AD0003E24A111A110A0130230BE000030A422B8
:100AE0001430F200F3013108F1003008F000BB22AD
:100AF0007408BC007508BD00E1231430F200F30156
:100B00003308F1003208F000BB227408BC007508FD
:100B1000BD00E1231430F200F3013508F100340880
:100B2000F000BB227408BC007508BD00E123A508D5
:100B3000031DA62DA408031DA62DA608031DA62D82
:100B400039083804031DA62DDC30A72DF030BC0079
:100B5000BD01E1231430F200F3013708F10036083B
:100B6000F000BB227408BC007508BD00E12304300E
:100B7000BC000130BD00E1231830BC000130BD00D5
:100B8000E1230330BE000030A4221430F200F30150
:100B90003108F1003008F000BB220A307407BC00B5
:100BA0000030031801307507BD00E1231430F20056
:100BB000F3013308F1003208F000BB220A30740759
:100BC000BC000030031801307507BD00E12314306C
:100BD000F200F3013508F1003408F000BB220A30BE
:100BE0007407BC000030031801307507BD00E12315
:100BF000A508031D072EA408031D072EA608031D24
:100C0000072E39083804031D072EE630082EFA3067
:100C1000BC00BD01E1231430F200F3013708F100FC
:100C20003608F000BB220A307407BC0000300318FD
:100C300001307507BD00E1230E30BC000130BD005E
:100C4000E1232230BC000130BD00E1239F2E0230A1
:100C5000BE000030A4222D307E232D307E232D3087
:100C60007E232D307E232D307E232D307E232D308C
:100C70007E232D307E232D307E232D307E232D307C
:100C80007E232D307E232D307E232D307E23033096
:100C9000BE000030A4222D307E232D307E232D3047
:100CA0007E230F307E233C307E2341307E2346302E
:100CB0007E234B307E2350307E230F30962E023021
:100CC000BE000030A4222D307E232D307E232D3017
:100CD0007E232D307E232D307E232D307E232D301C
:100CE0007E232D307E232D307E232D307E232D300C
:100CF0007E232D307E232D307E232D307E23033026
:100D0000BE000030A4222D307E232D307E232D30D6
:100D10007E232D307E232D307E230F307E233230F4
:100D20007E2337307E230F307E232D307E232D30DF
:100D30007E232D307E232D307E232D307E232303F2
:100D40000319BF2F2308023A0319872F8B13CC30C6
:100D50009F238B172119B32E8B1344309F238B179E
:100D60002115AD0121122119051EBD2E211EBD2EFA
:100D70008B13BE309F238B172114AE22211CFC2C19
:100D80008B13EA22A800EA22AA008B17BC002808CD
:100D90003E242112211121100530BE000030A42272
:100DA0001430F200F3013108F1003008F000BB22EA
:100DB0007408BC007508BD00E1231430F200F30193
:100DC0003308F1003208F000BB227408BC0075083B
:100DD000BD00E1231430F200F3013508F1003408BE
:100DE000F000BB227408BC007508BD00E123A50813
:100DF000031D062FA408031D062FA608031D062F9A
:100E000039083804031D062FDC30072FF030BC00F2
:100E1000BD01E1231430F200F3013708F100360878
:100E2000F000BB227408BC007508BD00E12304304B
:100E3000BC000130BD00E1231830BC000130BD0012
:100E4000E1230630BE000030A4221430F200F3018A
:100E50003108F1003008F000BB220A307407BC00F2
:100E60000030031801307507BD00E1231430F20093
:100E7000F3013308F1003208F000BB220A30740796
:100E8000BC000030031801307507BD00E1231430A9
:100E9000F200F3013508F1003408F000BB220A30FB
:100EA0007407BC000030031801307507BD00E12352
:100EB000A508031D672FA408031D672FA608031D9F
:100EC000672F39083804031D672FE630682FFA3082
:100ED000BC00BD01E1231430F200F3013708F1003A
:100EE0003608F000BB220A307407BC00003003183B
:100EF00001307507BD00E1230E30BC000130BD009C
:100F0000E1232230BC000130BD00E123FC2C053080
:100F1000BE000030A4222D307E232D307E232D30C4
:100F20007E232D307E232D307E232D307E232D30C9
:100F30007E232D307E232D307E232D307E232D30B9
:100F40007E232D307E232D307E232D307E230630D0
:100F5000BE000030A4222D307E232D307E232D3084
:100F60007E230F307E233C307E2341307E2346306B
:100F70007E234B307E2350307E230F30F62F0530FA
:100F8000BE000030A4222D307E232D307E232D3054
:100F90007E232D307E232D307E232D307E232D3059
:100FA0007E232D307E232D307E232D307E232D3049
:100FB0007E232D307E232D307E232D307E23063060
:100FC000BE000030A4222D307E232D307E232D3014
:100FD0007E232D307E232D307E230F307E23323032
:100FE0007E2337307E230F307E232D307E232D301D
:100FF0007E232D307E232D307E232D307E23FC2C2E
:02400E003C3F35
:00000001FF
